:100000000C945B000C9407020C9434020C94830053
:100010000C9483000C9483000C9483000C94830054
:100020000C9483000C9483000C9483000C94830044
:100030000C9483000C9483000C9483000C94830034
:100040000C9461020C9483000C9467040C9483005C
:100050000C9483000C9483000C9483000C94830014
:100060000C9483000C948300000024272A000025B0
:10007000282B000023262904040404040404040299
:100080000202020202030303030303010204081035
:100090002040800102040810200102040810200002
:1000A0000000070002010000030406000000000039
:1000B00000000000E30011241FBECFEFD4E0DEBF3C
:1000C000CDBF11E0A0E0B1E0E0E2FAE002C00590AF
:1000D0000D92AC30B107D9F711E0ACE0B1E001C04E
:1000E0001D92A33AB107E1F710E0C6EBD0E004C0DF
:1000F0002297FE010E940A05C43BD107C9F70E945E
:10010000DC000C940E050C9400008DE091E00E9440
:10011000F1008823B9F18DE091E00E94EE00809318
:100120000C01992787FD9095A92FB92F20E030E089
:10013000AC01BD018DE091E00E94F2016FEF70E033
:1001400089E00E9435036FEF70E08AE00E9435037A
:100150006FEF70E08BE00E9435036AE070E080E0B2
:1001600090E00E94D10260E070E089E00E943503D7
:1001700060E070E08AE00E94350360E070E08BE0B0
:100180000E94350308950F931F930DE011E040E89E
:1001900055E260E070E0C8010E94F40064E670E09F
:1001A00080E090E00E94D10260E071E0C8010E940E
:1001B00028011F910F9108950E94FB020E94C30025
:1001C0000E948500FDCF89E091E090930E0180931D
:1001D0000D010895862F0E942F0408950E9448045F
:1001E00008950E9437040895CB01BA010E94F603D6
:1001F00008950F931F93CF93DF938C01EB0109C0F8
:100200002196D801ED91FC910190F081E02DC8017B
:10021000099568816623A1F7DF91CF911F910F9116
:1002200008950F931F938C01DC01ED91FC910190D7
:10023000F081E02D6DE00995D801ED91FC910190E0
:10024000F081E02D6AE0C80109951F910F91089592
:100250000F931F938C010E94F900C8010E941101A5
:100260001F910F9108952F923F924F925F926F923C
:100270007F928F929F92AF92BF92CF92DF92EF9236
:10028000FF920F931F93DF93CF93CDB7DEB7A09765
:100290000FB6F894DEBF0FBECDBF1C016A017B0113
:1002A000411551056105710549F4DC01ED91FC91A1
:1002B0000190F081E02D60E3099554C088249924D1
:1002C0005401422E55246624772401E010E00C0FDF
:1002D0001D1F080D191DC701B601A30192010E943F
:1002E000B704F80160830894811C911CA11CB11C07
:1002F000C701B601A30192010E94B704C901DA0146
:100300006C017D01C114D104E104F104F1F681E036
:10031000E82EF12CEC0EFD1EE80CF91C3E010894B1
:10032000611C711CD501C4010197A109B1096C01BF
:10033000C818D90814C0F601EE0DFF1D60816A309F
:1003400010F4605D01C0695CD101ED91FC910190F8
:10035000F081E02DC10109950894E108F1086E14BF
:100360007F0449F7A0960FB6F894DEBF0FBECDBF4D
:10037000CF91DF911F910F91FF90EF90DF90CF9081
:10038000BF90AF909F908F907F906F905F904F90B5
:100390003F902F900895EF92FF920F931F93CF936A
:1003A000DF93EC017A018B0177FF0FC0E881F981BF
:1003B0000190F081E02D6DE2099510950095F09483
:1003C000E094E11CF11C011D111D2AE0B801A701F8
:1003D000CE010E943301DF91CF911F910F91FF90C9
:1003E000EF900895DC012115310541F4ED91FC9168
:1003F0000190F081E02D642F099508952A30310590
:1004000019F40E94CB0108950E94330108951F92B0
:100410000F920FB60F9211242F933F934F935F9338
:100420006F937F938F939F93AF93BF93EF93FF93BC
:1004300080910F0190911001892B29F0E0910F011B
:10044000F09110010995FF91EF91BF91AF919F91AC
:100450008F917F916F915F914F913F912F910F906D
:100460000FBE0F901F9018951F920F920FB60F920C
:1004700011242F933F934F935F936F937F938F93A9
:100480009F93AF93BF93EF93FF938091110190914E
:100490001201892B29F0E0911101F09112010995C7
:1004A000FF91EF91BF91AF919F918F917F916F914C
:1004B0005F914F913F912F910F900FBE0F901F9022
:1004C00018951F920F920FB60F9211242F938F93AE
:1004D0009F93AF93BF938091130190911401A091CA
:1004E0001501B09116010196A11DB11D8093130154
:1004F00090931401A0931501B093160180911701F8
:1005000090911801A0911901B0911A018050904C5E
:10051000AF4FBF4F8093170190931801A09319011B
:10052000B0931A0127C08091170190911801A091F2
:100530001901B0911A0180589E43A040B0408093A9
:10054000170190931801A0931901B0931A0180919B
:100550001B0190911C01A0911D01B0911E010196FB
:10056000A11DB11D80931B0190931C01A0931D013F
:10057000B0931E018091170190911801A09119016B
:10058000B0911A0181589E43A040B04060F6BF91DF
:10059000AF919F918F912F910F900FBE0F901F9051
:1005A0001895EF92FF920F931F937B018C018FB7E9
:1005B000F89440911B0150911C0160911D017091B4
:1005C0001E018FBF2FB7F89480911B0190911C01E1
:1005D000A0911D01B0911E012FBF841B950BA60B8E
:1005E000B70BE816F9060A071B0760F71F910F9172
:1005F000FF90EF900895789484B5826084BD84B5AF
:10060000816084BD85B5826085BD85B5816085BD0D
:10061000EEE6F0E0808181608083E1E8F0E08081B7
:1006200082608083808181608083E0E8F0E0808167
:1006300081608083E1EBF0E0808184608083E0EB87
:10064000F0E0808181608083EAE7F0E0808184606F
:1006500080838081826080838081816080838081CB
:10066000806880831092C10008951F93CF93DF9319
:10067000182FEB0161E00E948D03E12FF0E0E156BD
:10068000FF4F8491833051F4809180008068809383
:100690008000D0938900C09388003BC0843051F41F
:1006A00080918000806280938000D0938B00C09303
:1006B0008A002FC0813039F4209729F184B58068F1
:1006C00084BDC7BD26C0823039F42097E1F084B5DF
:1006D000806284BDC8BD1DC0863041F48091B000E9
:1006E00080688093B000C093B30013C0873041F49A
:1006F0008091B00080628093B000C093B40009C0C4
:10070000C038D10514F460E001C061E0812F0E947F
:10071000AB03DF91CF911F910895282F30E0C901DD
:1007200085579F4FFC01949129583F4FF9018491BF
:10073000882381F0E82FF0E0E859FF4FE491F0E0E2
:10074000662329F480819095892380830895808190
:10075000892B80830895482F50E0CA0181569F4F0E
:10076000FC012491CA0185579F4FFC01949149587F
:100770005F4FFA0134913323C1F1222331F1233049
:1007800021F4809180008F7705C0243031F480916E
:1007900080008F7D8093800018C0213019F484B5CB
:1007A0008F7704C0223021F484B58F7D84BD0DC0C5
:1007B000263021F48091B0008F7705C0273029F4CE
:1007C0008091B0008F7D8093B000E32FF0E0E3597B
:1007D000FF4FE491F0E0662329F48081909589230E
:1007E000808308958081892B80830895EF92FF9202
:1007F0000F931F937B018C0122E030E040E050E03A
:100800000E94D904205C3D4B404F5F4FCA01B901A3
:10081000A80197010E94D904C901DA010197A10931
:10082000B109292F3A2F4B2F552747FD5A9501968D
:10083000A11DB11D2093C50081508093C400E1EC3F
:10084000F0E0808180618083808188608083808106
:10085000806880831F910F91FF90EF900895982FEB
:100860008091C00085FFFCCF9093C60008958091D1
:100870001F019091200180589F4F209121013091BC
:100880002201821B930B60E870E00E94A40408958B
:10089000409121015091220180911F0190912001EE
:1008A0008417950719F42FEF3FEF0FC0FA01ED5DA4
:1008B000FE4F2081CA01019660E870E00E94A40406
:1008C000909322018093210130E0C90108951F9285
:1008D0000F920FB60F9211242F933F934F935F9374
:1008E0006F937F938F939F93AF93BF93EF93FF93F8
:1008F0004091C600E0911F01F0912001CF010196C7
:1009000060E870E00E94A4049C0180912101909114
:1009100022012817390739F0ED5DFE4F40833093EF
:10092000200120931F01FF91EF91BF91AF919F9103
:100930008F917F916F915F914F913F912F910F9088
:100940000FBE0F901F90189597FB092E07260AD00F
:1009500077FD04D049D006D000201AF47095619537
:100960007F4F0895F6F7909581959F4F0895A1E2E6
:100970001A2EAA1BBB1BFD010DC0AA1FBB1FEE1F19
:10098000FF1FA217B307E407F50720F0A21BB30B64
:10099000E40BF50B661F771F881F991F1A9469F7E0
:1009A00060957095809590959B01AC01BD01CF013C
:1009B000089597FB092E05260ED057FD04D0D7DFEA
:1009C0000AD0001C38F450954095309521953F4F42
:1009D0004F4F5F4F0895F6F790958095709561950C
:1009E0007F4F8F4F9F4F0895AA1BBB1B51E107C03C
:1009F000AA1FBB1FA617B70710F0A61BB70B881FAF
:100A0000991F5A95A9F780959095BC01CD0108953D
:100A1000EE0FFF1F0590F491E02D0994F894FFCF9D
:0C0A2000486F6C610000000000EA00005C
:00000001FF
